:020000001028C6
:0200080042288C
:10002000FF309A009B009B0B13289A0B1328850125
:1000300086018316850105150516860106148614AA
:10004000061601178116011281110110811001118C
:1000500083120B160730990064309C0005080439A0
:1000600013069500151D2E28050804399300131951
:100070002E28181C3D2818102E2881010B118B10DA
:100080008B172E289700030E9600831601158114F6
:1000900001148312990B522807309900861500002D
:1000A0000000861100308C008D008E000B1D5F2833
:1000B00002308C0005308D0006308E000B11811F40
:1000C000682801308F000230900008309100A8208D
:1000D000011F712800308F0006309000043091001D
:1000E000A820811E7A2800308F0003309000023053
:1000F0009100A820011E832800308F00013090005D
:1001000006309100A820811D8C2800308F0000301F
:10011000900008309100A820011D952800308F0024
:100120000030900004309100A820811C9E280030EF
:100130008F000030900002309100A820011CC128DF
:1001400000308F000030900001309100A820C128BD
:1001500003010E0711078E00F63E031CB2288D0A1C
:100160000A308E0203010D0710078D00F63E031CB6
:10017000BC288C0A0A308D0203010C070F078C0083
:1001800008008C1CD2280C1CD2280D1DD2288D1CD6
:10019000D2288C018D018E01D22830308E048D043E
:1001A0008C0408001D18D528DC2886123E218616EE
:1001B0003E2102309D0044298618EE289E0A1E1D0D
:1001C00044299E1E44291E1F442900309F00A00080
:1001D000A10000309E0001309D00442901309D00A7
:1001E00000309E003E2106113E219F01A001A10189
:1001F00025212521252125212521252125219F0076
:1002000025219F0D1F109F042521A00D2010A00463
:100210002521A00D2010A0042521A00D2010A00450
:100220002521A00D2010A0042521A10D2110A1043D
:100230002521A10D2110A1042521A10D2110A1042A
:100240002521A10D2110A1043B290F30A200A20BF2
:10025000272906130F30A200A20B2C290617000035
:10026000000000000608A300A30CA30CA30CA30C21
:1002700023080139080006153E2144291030A40046
:10028000B321A40B40290800210891002008900008
:100290001F088F00A8200C08FC3E031857290C08E3
:1002A000FD3E031C69290D08FA3E031C69290D084F
:1002B000FA3E8D00031865298D038D038D038D0390
:1002C0008D030D030F398D008C038C038C038C037D
:1002D0006929CD20253092008C210C0892008C21B8
:1002E0000D0892008C210E0892008C212F30920074
:1002F0008C21373092008C210D3092008C21181403
:1003000064309C0083160111811001108312160EB7
:100310008300970E170E0800AD21121CAD21121894
:10032000B021921CAD219218B021121DAD211219DD
:10033000B021921DAD219219B021121EAD21121AC9
:10034000B021921EAD21921AB021121FAD21121BB5
:10035000B021AD21B021B02108008511B3210800E2
:100360008515B3210800F0309400940BB5290800DE
:00000001FF
